:020000020000FC
:100000000AC018951895189518951895189518956B
:100010001895189518950FED0DBF0AEA07BB0CE36C
:1000200001BB08E10AB906E003B900E002B90AE041
:1000300009B900E002BB02D10D34D9F700E002BBE0
:10004000FDD00433B1F7929AF9D0073691F7939A1D
:10005000F5D0013371F7949AF1D0033651F7EED011
:10006000959A013231F71124222433244424552453
:100070006624772488249924AA24BB24CC245F995D
:100080005DC010E0929800E8AFD0031710F0116047
:10009000929A939800E2A8D0041710F01260939AF5
:1000A000949808E0A1D0051710F01460949A9598E0
:1000B00002E09AD0061710F01860959A272F712F3A
:1000C0002127212310E001E020FF03C0100E211E94
:1000D000311E21FF03C0400E511E611E22FF03C0CE
:1000E000700E811E911E23FF03C0A00EB11EC11E03
:1000F000C6CF012D9FD0022D9DD0032D9BD0042D66
:1001000099D0052D97D0062D95D0072D93D0082D89
:1001100091D0092D8FD00A2D8DD00B2D8BD00C2D89
:1001200089D011242224332444245524662477249E
:1001300088249924AA24BB24CC24A1CF0CB1073451
:10014000C1F2043771F00435A9F00235E1F003344F
:1001500039F1013219F00FE36DD091CF0EE76AD07B
:100160008ECF032F67D0042F65D0052F63D0062FC5
:1001700061D085CF63D0302F61D0402F5FD0502F1A
:100180005DD0602F7CCF00E82FD054D000E22CD07F
:1001900051D008E029D04ED002E026D04BD06FCF0E
:1001A0004DD010E0013309F410E8023309F410E2F5
:1001B000033309F418E0043309F412E0103099F025
:1001C000012F10E02FEF0F930FD0011708F0102F21
:1001D000021708F4202F0F915F9BF5CF0CB1012F70
:1001E00029D0022F27D04BCF1F932F93202F102FD2
:1001F0000695102B17BB00E008BB00E000000A9535
:10020000E9F727BB00E008BB0FEF03950F3F61F054
:10021000023310F011E401C014E11A95F1F716B39E
:10022000110F1223103089F310E017BB18BB2F9168
:100230001F9108955D9BFECF0CB908955F9BFECF83
:040240000CB1089560
:00000001FF
